:10000000FC7F0020E9050000D5050000D9050000AF
:1000100000000000000000000000000000000000E0
:10002000000000000000000000000000DD050000EE
:100030000000000000000000E1050000E5050000F0
:1000400010B5064C2378002B07D1054B002B02D0AE
:10005000044800E000BF0123237010BD5C000020B5
:10006000000000009817000008B5084B002B03D0D3
:100070000748084900E000BF07480368002B03D089
:10008000064B002B00D0984708BDC046000000007A
:1000900098170000600000205800002000000000B9
:1000A00010B5C3699C07FCD403680224A343036012
:1000B000C46901231C42FBD1046823430360036825
:1000C000DC07FCD4C46901231C42FBD1C469DC40B9
:1000D0001C42F7D1084B1A430260C3695A07FCD48B
:1000E000C0239B0243608181C3699C07FCD40368E1
:1000F00002221343036010BD04000040037EDA07B0
:10010000FCD5018570470000027E01235107FBD515
:10011000428B1A4207D1428BDA401A4203D1428BFA
:1001200092081A4202D0034B01221A70008DC0B20D
:100130007047C0467800002070B50368041C988B97
:100140001A1C0821FF32084228D0988B174D014312
:10015000802099839872112353704021144B917120
:1001600050715E68C0202E40800506435E605E6967
:100170003540284358610F4818600F4818615D6882
:100180000E4828408025AD02284358605868800BEF
:100190008003586000235171237105E0137ADA0659
:1001A00002D5201C00F0EEFA207970BDFFFFFF8F12
:1001B000940100209400002014010020FF3F00F073
:1001C000002303714371044B016083600B780222AA
:1001D00013430B707047C0463901000038B5364BE9
:1001E0002021DA6901200A43DA61344B06241A78A7
:1001F00002431A70324B0F22197891431970197803
:10020000214319702F490C782043087019780A404F
:100210001A701A7860210A431A702B4B2B4A5A80A5
:100220005A7852B2002AFBDB294B01211A780A4383
:100230001A709A78D107FCD426480268510B1F2205
:100240001140914200D1052111408C011D8D2249A0
:100250002940214319850468A10C0A401F2A00D1B6
:100260001D221C8D1F210A408C4322431A850268DF
:100270000721D20D0A408A4200D103220A40188D7C
:100280001103164A02400A431A8519787F220A4050
:100290001A701A78042112480A431A7058621A898F
:1002A0000C218A431A811A8901218A431A8100216B
:1002B000802201F006F938BD000400405844004196
:1002C0003C44004159440041000C004006400000FD
:1002D00000500041246080003FF8FFFFFF8FFFFFC8
:1002E00094010020F7B5141C234A5F0101971D1CDF
:1002F000D319061C5869271C4000400F03301033E7
:10030000C74006D00F1C8022596812060A435A6063
:1003100009E02F1C7B1E9F41184BBF01FF18381CA2
:10032000221C01F0C5F801991348083542181761DD
:10033000131C5269A104920B890C92030A435A615F
:1003400059690F4A02200A405A616B01F318D979A2
:10035000032211400143D8799043021C0A43DA7109
:100360005979802252420A435A716B01F318DB79A2
:100370009A07FAD5201CFEBD94010020140100202C
:10038000FF3F00F0F8B51E4E041C3378151C002BFF
:1003900012D11C4B1C4A1A645A6C920B92035A6479
:1003A000586C1A4A02405A64A2235B00E25C402067
:1003B0000243E254012333704827FF37E25D0123F3
:1003C00013401AD00F4B5A6C9204920CAA4202D2DC
:1003D0005D6CAD04AD0C081C2A1C0B4901F068F8DB
:1003E000E25D03231A4001210A43E15D99430B1C9E
:1003F0001343E3550023337000E01D1C281CF8BD97
:100400007900002094010020D4000020FF3F00F07C
:10041000FF30827930239A43131C2022002900D117
:1004200010221343837170470C4BFF305A6902212D
:10043000920B92035A61027A03231A400A43017A0B
:1004400099430B1C13430372827980235B4213434D
:100450008371037A9A07FCD57047C0469401002047
:1004600080235B421943C9B28172704770B5A023E3
:1004700003225B00C254134B134A5C6CC02114402E
:1004800089050C4346255C64FF35402444550F4DD7
:1004900030261D6490256D0046555D6B154029433F
:1004A000922559636D0080214155094D1D63B0258A
:1004B0006D0044555C6F22405A67B2235B00C15403
:1004C00070BDC04694010020FFFFFF8FD4000020C4
:1004D0005401002030B5364A1E2351680820994344
:1004E00002231943516033498A6902438A613248C1
:1004F000324A9082908A03439382D3689807FCD54E
:100500002F4B012018701878C40704D52C48407868
:1005100040B20028F7DB01209860587840B20028EC
:10052000FBDB284C26484460587840B20028FBDBAF
:1005300082242348E4014480587840B20028FBDB41
:10054000908C8024A0439084D068C506FCD51E4CB6
:100550001A48C462D4681948E506FBD5848C1B4D43
:100560002C438484D4681548E506FBD5848C022589
:100570002C438484D0680406FCD51048C068450626
:10058000F8D5D068C406FCD500229A605A7852B2D9
:10059000002AFBDB0E480A4A50605A7852B2002A01
:1005A000FBDB00230B724B728B72CB7230BDC046EB
:1005B00000400041000400400C060000000800401C
:1005C000000C004001050100B805FF7D040A000091
:1005D000000703000EBEFEE70DBEFEE705BEFEE708
:1005E00002BEFEE701BEFEE70E4A0F4838B5824262
:1005F00004D10E4A0E4B93420ED10AE00D4C9442A8
:10060000F7D00023D1188842F3D9E55804330D60A0
:10061000F8E700F04DF804E09342FAD2002102C35B
:10062000FAE7FEE7000000205C000020A0030020A5
:100630005C0000209C170000194A10B51188FA24AC
:10064000013189B2174BA400A14201D011801CE0F6
:1006500000211180144900240C5760431C880019A4
:1006600080B204B2FF2C01DC188002E0FF20188069
:1006700008700024185F002803DA00201880012089
:1006800008708020094980028861128800215B5E21
:100690009A4203D18022054B92025A6110BDC04696
:1006A0007A0000207C00002000000020004400416F
:1006B00038B580222B4B92029A605A612A4A1C1C40
:1006C000117801221140294B002200290AD1186813
:1006D000274A904201D1196018E01A60254A013A70
:1006E000002AFCD11A60244B1A68191C501C0DD02A
:1006F000D8B200280AD180208002A06182F3088845
:10070000FF2293431D4A93604B681847FFF7E2FEB0
:1007100062B600F0FBFC00F0CFF980239B02051CC1
:10072000A3610320FFF788FFAB68281C9847144B90
:10073000002801D001221A701A78002A05D0002062
:1007400000F036FA00F092FAFCE71B78002BE8D1B3
:1007500000F050FD0028E4D0012000F029FA00F05C
:1007600085FAFCE70044004138040040FC7F00208B
:100770003581730748E801000020000000ED00E02B
:100780007E000020F8B50468051C201CFF30037AA9
:10079000B64A10210B430372B54F1378B5493B702D
:1007A0005378B54E0B7093783380D1783388090233
:1007B0000B4333801179B14B198051791F8809029D
:1007C0000F431F809779AE490F80D2790F881202AC
:1007D0003A430A8040224271A648A54F02783878F1
:1007E000A84F12020243181CBA4200D199E01EDC45
:1007F000802149008A4200D158E107DC812A6AD071
:10080000822A6ED0802A00D050E164E081235B0010
:100810009A4200D1AFE000DA23E1C0239B009A4264
:1008200000D143E1984B9A4200D11AE13EE1902376
:100830001B019A4242D015DCD023DB009A4222D021
:1008400088231B019A4242D0A023DB009A4200D0A9
:100850002CE1201CFFF7E8FD3188286889B2FFF7FA
:10086000FFFD27E1894B9A4200D1FAE000DC1DE14F
:10087000874B9A4200D1E8E0864B9A4200D015E1BE
:1008800033886B71EDE033881B0A012B08D10B888C
:1008900012222868934201D80A8892B27E49DCE08D
:1008A00033881B0A022B00D000E10B884322286802
:1008B000934201D80A8892B27849CEE03388201C4E
:1008C0002B71FFF7B1FD201CFFF7D0FDF2E0291CD2
:1008D00001C90122C1E0724900230B80286802226D
:1008E000BCE06F4900220A801888502210406D4AEF
:1008F00010701E880F20304018801888032800D9F7
:10090000D4E012781B8808335B01E418A379002A2D
:1009100001D09B0600E0DB06DB0F0B80286802227B
:100920009BE019887F2291435E4AC9B211701888F2
:100930000F21014019803188002900D0B6E01988C4
:10094000002900D1B2E01988032900D9AEE012785D
:100950001B8808335B01E318002A05D05A7930213F
:100960008A4320210A4304E05A7930218A43102027
:1009700002435A7175E002887F239A43494BD2B2F1
:100980001A7001880F220A4002803288002A00D0A3
:100990008CE00288002A00D188E00288032A00D96E
:1009A00084E01B78002B27D0038808335B01E31811
:1009B0009B79990655D50388302108335B01E318EC
:1009C0001A798A4320210A431A71038808335B018C
:1009D000E318DB795A0644D50388602108335B01AC
:1009E000E318DA798A4340210A43DA710388022244
:1009F00008335B01E31826E0038808335B01E31842
:100A00009B79DF062DD50388302108335B01E3187D
:100A10001A798A4310210A431A71038808335B014B
:100A2000E318DB7999061CD50388602108335B0144
:100A3000E318DA798A4320210A43DA710388012214
:100A400008335B01E3181A710BE00B880822286851
:100A5000934201D80A8892B213490023FFF742FC5F
:100A600028E0201CFFF7E0FC24E0C04694000020B2
:100A7000890000207F0000208000002084000020EA
:100A80008600002002030000010300002120000076
:100A9000A121000021220000EC140000040000202D
:100AA000820000208800002048000020201C012136
:100AB000FFF7AEFCF8BDC04610B5054B054C2360F2
:100AC000FFF78CFB201C2168FFF77AFB201C10BD70
:100AD000005000411402002007B5054B012201908F
:100AE00001A91868131CFFF7FDFB01200EBDC046CD
:100AF0001402002013B5054B6C4607341868211CFE
:100B00000122FFF73FFC207816BDC04614020020EA
:100B100010B5074C201CFFF70FFB031C002083427D
:100B200005D022684823FF33D05C0123184010BD54
:100B30001402002010B5054A0C1C031C191C106877
:100B40000123221CFFF7CEFB201C10BD1402002045
:100B500070B5084C061C201C0D1CFFF7EDFA002395
:100B6000984205D02068311C2A1CFFF70BFC031C9F
:100B7000181C70BD14020020F8B50C4C051C201C7C
:100B80000E1CFFF7D9FA0023271C341C98420AD008
:100B9000002C07D0291C221C3868FFF7F3FB241A0D
:100BA0002D18F5E7331C181CF8BDC04614020020B0
:100BB000012805D1054B064A1A60064B187004E05F
:100BC000002802D1044A014B1A60704784020020B9
:100BD00020150000910000206C15000030B51A4B64
:100BE00085B01B78002B29D0042901D1026804E0CC
:100BF000022901D1028800E00278490004A84318C4
:100C00000B3B5C1AA3420BD00F201040092802D8DE
:100C10003025284300E0373018701209013BF1E716
:100C200001A830230370782343700A2243189A7076
:100C30000D22DA70054B04311B6801E0034B1B6881
:100C4000DB68984705B030BD90000020840200208A
:100C500072B6EFF30883044A1360036883F30888CD
:100C6000436818477047C04688020020F0B58FB02F
:100C700006A9CE4A0B1C31CA31C351CA51C360CA3E
:100C800060C3CB4CCB48A3687A255B035B0F9B000A
:100C90005B58C9490360A26892B253430A60C749CE
:100CA000C74A0B6000231360C64B1D700320FFF77B
:100CB000C3FCC54BC54D1B68281C1B6940219847C8
:100CC000C34B00221860C34B1D60C34BC24DC04FC5
:100CD0001A60286839688842E8D2BE4B1B681A78C7
:100CE000FF2A00D1F6E1232A00D0CDE1BB4E3378B4
:100CF000002B05D0B44BBA481B680221DB6898472B
:100D0000B04B1B78532B38D13B682A6893421ED9CD
:100D1000B04801322A609A1AB24B01681B6801314F
:100D20000160B14E9A4201D2326000E03360A448C3
:100D300032680068029000F0BBFB336829685A18DB
:100D40002A60A44A1668F1181160A84A13702B682B
:100D5000013B2B609F4B1A68013A1A60A34BA14AD2
:100D60001B7811688B4206D2974A95481268006832
:100D7000C91A92699047C04675E1522B07D1904A33
:100D8000914B10681B68974A5B6911686AE14F2BA9
:100D900005D18B4B934A1B6812681A7063E1482B8C
:100DA00005D1874B8F4A1B6812681A805BE1572B6D
:100DB00005D1834B8B4A1B6812681A6053E16F2B75
:100DC00003D17F4B0121186807E0682B08D17C4BC9
:100DD00084481B6802211B880360FFF7FFFE42E185
:100DE000772B06D1764B7F481B6804211B68036074
:100DF000F3E7472B13D17B4B1868FFF729FF7C4B98
:100E00001B6883F3088862B67A4B1B78002B00D1ED
:100E100029E16D4B06201B681B68984723E1542B82
:100E200004D101233370684B1B685CE04E2B0BD15F
:100E30003378002B05D1644B69481B680221DB68BD
:100E40009847002333700EE1562B50D15E4D01219F
:100E50002B686948DB6898472B680321DB68674883
:100E60009847674E2B68301CDB68012198472B6838
:100E70000D21DB68634898472B68301CDB68012133
:100E80009847544F604B544E3B60002333603A1CEC
:100E9000311C1368581C10601B780393002B03D07F
:100EA0000B6801330B60F4E72B683168DB68564848
:100EB00098472B685248DB680121984703983060B7
:100EC00052483860434A1368591C11601A78424BE3
:100ED000002A03D01A6801321A60F3E72A681968F9
:100EE000D36898472B68DB683D480221BAE03D4A49
:100EF000582B15D12F4E314D366813682A68B10032
:100F0000934208D25808E06141482080207DC507FF
:100F1000FCD55B18F4E72C4B3E481B68DB68A0E06F
:100F2000592B33D11268264B3B49002A02D11B684A
:100F30000B6026E00868196863688025AB43920857
:100F40006360002A1DD0354B2380237DDE07FCD54E
:100F50000023184D2D680095AD08AB4202D3304DEB
:100F6000258006E09342FAD09D00465901334E5148
:100F7000EFE7257DEE07FCD59D0049194019D21AEF
:100F8000DFE7114B27481B68DB686AE05A2B6AD100
:100F90000B4B17681D680026EF19BD4244D0287816
:100FA000311C00F049F90135061CF6E70015000078
:100FB000004000413C0200203402002030020020AA
:100FC000800200202C020020840200204002002029
:100FD0002402002028020020380200209000002077
:100FE000601500008C0200209002002020020020EA
:100FF00088020020910000203C15000065150000CB
:101000003E15000088150000401500004C1500003A
:1010100002A5FFFF551500008C00002044A5FFFF2E
:1010200004A5FFFF591500002E4D2F482B68012104
:10103000DB68984707230F223240111C36093031F4
:10104000092A00DD07311020C0186A468154013B8F
:10105000F1D22B6804A8DB68082198472B68234845
:10106000DB6803219847224D7A232B70214B002205
:101070001A60214B1B7893422CD01A4B01211B681C
:101080001E48DB68984725E0111C3039C8B2194B5F
:10109000092804D81E683201114319601AE0111C96
:1010A0004139052903D81868373A010106E0111CB7
:1010B0006139052904D81D68573A29010A4308E017
:1010C0002C2A03D10E4A1E68166001E008490A70F6
:1010D00000221A600B4B1A6801321A600A4B1A6818
:1010E0000132F3E5840200205D1500005F15000069
:1010F0002C0200208C0200209000002063150000CC
:1011000080020020380200202802002010B51C4B6D
:1011100001201A78022402431A701A4B0F22197800
:101120009143197019782143197017490C7820439D
:10113000087019780A401A701A7820210A431A7028
:10114000124B04211A6A0A431A62114B114A5A803F
:101150005A7852B2002AFBDBC4220F480F4992038F
:10116000FEF79EFF0E4A002313700E4A13700E4ABC
:1011700013700E4A13700E4A13700E4A137010BD8E
:101180004A440041354400414B44004100040040C2
:10119000000C004014400000000800422AF6000045
:1011A000940200201B0300209502002098020020DA
:1011B0001C0300201903002008B5C1B20248FEF745
:1011C0009DFF012008BDC04600080042024B187E6A
:1011D0004007C00F7047C0460008004208B5FFF73F
:1011E000F5FF0028FBD00248FEF78EFF08BDC04681
:1011F0000008004208B5FFF7E9FF0023984205D038
:10120000FFF7ECFF031C233B5A425341181C08BD57
:1012100070B5041C0D1C4618B44204D02078FFF7AA
:10122000CBFF0134F8E7281C70BD10B5041CFFF794
:10123000D5FF2070012010BD0B0A5840034B400021
:10124000C05A0902484080B27047C0469615000057
:10125000F7B50024051C0F1C261CBC4220D0FFF74C
:10126000BDFF114BC0B21B780190002B1AD1311C6D
:10127000FFF7E2FF0D4B061C1A88002A04D10C4A26
:1012800011782A1C002907D001996A1C2970802F27
:1012900002D11988013919800134A4B2151CDCE788
:1012A000301C00E00120FEBD190300209602002042
:1012B0001A030020F0B53E4E85B0002203900C1CAE
:1012C00032703C4B914201D1012201E03A490C803D
:1012D0001A707F231C4201D080349C43FFF77EFFAD
:1012E0003378C0B2002B07D000253570FFF776FFAA
:1012F0003378C0B2AB4236D1432803D0712853D0E3
:101300001528EBD1012300930120FFF755FF00982A
:10131000FFF752FF00998025C843C0B2FFF74CFF8A
:10132000039B00270293244A1388002B1DD12149D7
:1013300001930978002918D10198FFF73DFF391C66
:101340000198FFF779FF013D071C002DEBD1000A42
:10135000C0B2FFF731FFF8B2FFF72EFFFFF73EFFF5
:101360003378002B0AD035701FE00299013B0978D1
:101370001380029B019101330293DDE7C0B206287E
:1013800007D1009B03990133DBB280310093803C8D
:101390000391002CB8D10420FFF70EFFFFF71EFFCA
:1013A000044B01251C7000E00025281C05B0F0BD91
:1013B000190300201A03002096020020F0B5384CD3
:1013C00087B0002301902370994201D1012301E0ED
:1013D000344A1180344A642613704320FFF7ECFE30
:1013E000324FFFF7F3FE002803D1002F03D0013F57
:1013F000F7E7002F03D1013E002EEED14DE001258D
:10140000FFF7ECFE2378002B38D1C0B20290012800
:1014100005D004283DD10620FFF7CEFE39E005AE09
:101420000221301CFFF714FF01988021FFF710FF05
:1014300023780390002B18D1FFF7D0FE0702FFF7A7
:10144000CDFEBFB223783F18BFB2012B0DD0039B56
:101450009F4207D13378AB4204D1EB437278DBB2C1
:101460009A4204D01820FFF7A7FE002303E00620CD
:10147000FFF7A2FE029B2278002A02D000262670E7
:101480000BE0012B05D1019A6B1C8032DDB2019279
:10149000B6E7054A002313700126301C07B0F0BDE3
:1014A00019030020960200201A03002000350C00CA
:1014B00010B50023934203D0CC5CC4540133F9E748
:1014C00010BD031C8218934202D019700133FAE751
:1014D00070470000F8B5C046F8BC08BC9E4670478F
:1014E000F8B5C046F8BC08BC9E4670471201000221
:1014F000020000409A230B000002000000010000DF
:101500000800000010000000200000004000000063
:101510008000000000010000000200000004000044
:10152000B9110000DD110000CD1100001112000002
:101530002B120000B5120000BD1300007600200041
:101540004D617220203520323031360031373A3447
:10155000363A353200580A0D00590A0D005A002358
:101560000A0D003E00322E3000000000D90A0000B3
:10157000F50A0000110B0000350B0000510B0000B4
:10158000350B0000790B00005B41726475696E6F6A
:101590003A58595A5D0000002110422063308440BF
:1015A000A550C660E770088129914AA16BB18CC132
:1015B000ADD1CEE1EFF13112100273325222B552A9
:1015C0009442F772D662399318837BB35AA3BDD382
:1015D0009CC3FFF3DEE36224433420040114E66479
:1015E000C774A44485546AA54BB528850995EEE5D2
:1015F000CFF5ACC58DD55336722611163006D77689
:10160000F6669556B4465BB77AA719973887DFF721
:10161000FEE79DD7BCC7C448E5588668A778400850
:10162000611802282338CCC9EDD98EE9AFF9488971
:1016300069990AA92BB9F55AD44AB77A966A711AE8
:10164000500A333A122AFDDBDCCBBFFB9EEB799BC1
:10165000588B3BBB1AABA66C877CE44CC55C222C38
:10166000033C600C411CAEED8FFDECCDCDDD2AAD11
:101670000BBD688D499D977EB66ED55EF44E133EC8
:10168000322E511E700E9FFFBEEFDDDFFCCF1BBF61
:101690003AAF599F788F8891A981CAB1EBA10CD13B
:1016A0002DC14EF16FE18010A100C230E320045043
:1016B000254046706760B9839893FBA3DAB33DC3B6
:1016C0001CD37FE35EF3B1029012F322D232354293
:1016D000145277625672EAB5CBA5A89589856EF546
:1016E0004FE52CD50DC5E234C324A01481046674E3
:1016F000476424540544DBA7FAB79987B8975FE796
:101700007EF71DC73CD7D326F2369106B016576632
:101710007676154634564CD96DC90EF92FE9C8991D
:10172000E9898AB9ABA94458654806782768C01882
:10173000E1088238A3287DCB5CDB3FEB1EFBF98BF5
:10174000D89BBBAB9ABB754A545A376A167AF10AD2
:10175000D01AB32A923A2EFD0FED6CDD4DCDAABD05
:101760008BADE89DC98D267C076C645C454CA23C22
:10177000832CE01CC10C1FEF3EFF5DCF7CDF9BAFD5
:10178000BABFD98FF89F176E367E554E745E932E72
:10179000B23ED10EF01E000000000000010000006B
:1017A0000902430002010080320904000001020224
:1017B0000000052400100104240200052406000195
:1017C0000524010001070583030800FF0904010047
:1017D000020A00000007058102400000070502021E
:1017E0004000000000C20100000008006900000085
:1017F0004100000000000000FFFFFFFFFFFFFFFFB0
:10180000FFFFFFFFFFFFFFFFFFFFFFFFFFFFFFFFE8
:10181000FFFFFFFFFFFFFFFFFFFFFFFFFFFFFFFFD8
:10182000FFFFFFFFFFFFFFFFFFFFFFFFFFFFFFFFC8
:10183000FFFFFFFFFFFFFFFFFFFFFFFFFFFFFFFFB8
:00000001FF
